BPM For-Each Block

Hello all,
      My scenario works like JDBC - XI - JDBC. I will get se of rows from Database I have to send each row to update target field using For-each block in BPM. Here I will be using Synchronous send to JDBC so that if the data gets updated I'll get update_count as response. My doubt is consider i'm having 5 rows i'm passing each row into the for-each block two messages successfully updated third row is throwing some SQL exception at this time is it possible for me to catch this error? Also bcoz of this exception the rest of the rows  should not be affected. Please help me regarding this regard.
Best Regards,
Raj.

Hi,
You can try this.
After the send step in the BPM, use a container step to assign the response from the JDBC to a multiline container.
Then you will have all the responses for the individual rows. Whenever the no. of records updated is 0, you can take appropriate action.
Regards,
Puloma.

Similar Messages

  • BPM for each block doubt

    Hi guys,
    I'm doing a scenario where i'm using multi mapping transformation to populate two different RFC's and both of these RFC's are populated multiple times
    i.e. my source strucrure causes generation of multiple messages in my two RFC's
    After the transformation step, if i'm correct i need to use a block for each step
    Can anyone help me with the configuration on the for each block i.e. the value i need to enter for Curren Line and End condition.
    For multiline element, i think i need to use my multiline container object for the RFC source structure created by  transformation
    Thanks guys
    Varun

    You dont need to create the multi line container. Instead of that adopt MultiCast-ForEach Pattern.) This may solve your problem.
    In the BPM you define the following steps
    Start
    Receive Msg
    Dynamic Sequential Processing
       Send Msg
        Receive Msg
        Loop Sequentially(Multicast-ForEach)
    Stop
    The block is defined as a ForEach. Within the block a send step sends the msg to the first receiver in the receiver list and creates the correlation Correleation. A recever step user correalation and receives the response msg from the first receiver. If this receive step is complete the msg is send to next receiver list.

  • Indivdual Drill Filters for each Block

    Hello,
    Is it possible to have individual Drill Filters for each block of a report in BO XI R2? Suppose i have a Cross tab report and graph in the same report, and i want to apply individual Drill FIlters for Cross Tab Report and Graph. Can we do this in BO XI R2?

    You can use for Block1  the objects from the first query only.
    For example:
    =[Query1].[Region]
    and for block2 you use the merged dimension:
    =[Region]
    If it doesn't work you can try this other way of solving it (check this link):
    restrict drill downs in two blocks
    Edited by: PadawanGirl on Jan 19, 2011 5:53 PM

  • GarageBand - How to set different BPM for each track?

    Hi, for the last couple of years, I've been using Sony Acid on my PC to mix multiple tracks to make blends and remixes of songs. I've just switched of the a MacBook, and am trying to get Garage Band to do the same. I'm curious whether or not I can set the BPM of each track individually so they will all play at the same BPM when mixed. I'm only able to find the master BPM that changes the entire BPM. Any help would be great. Thanks in advance.

    Well, as far as I can see you don't really want different BPMs on each track, but you want all tracks to have the same tempo - only you want to make the tracks fit that tempo.
    You could do that in GB by first bringing each of the tracks to the desired tempo, then export it and re-import it. (There's some other ways to do it, but they all involve some fiddling around and maybe some math.*)
    Logic offers a nice feature where you can shorten and lengthen a region just by dragging it out. That could be used for the purpose you're trying to achieve.
    *For example: Determine the BPM of each of the tracks. Set the project's tempo to the BPM of track A. Import track A, turn it purple so it follows the tempo. Then set the project to project B's tempo, import it, etc. You will end up with all tracks in the same tempo, and you can still make the whole project go faster or slower.

  • BPM Message Split in Block par for Each: Just last message is sent n-times

    Hello everybody,
    we got BPM with a message split. In a par-for-each block the message is send.
    Asuming I have 3 lines in the multiline container element, I can see in SXMB_MONI that that message is send 3 times.
    The error is, that 3 times the last message is send.
    <u>Sample Error:</u>
    Message incoming in BPM:
    <root>
      <mymessage>M1</mymessage>
      <mymessage>M2</mymessage>
      <mymessage>M3</mymessage>
    </root>
    Messages outgoing:
    <root>
      <mymessage><b>M3</b></mymessage>
    </root>
    <root>
      <mymessage><b>M3</b></mymessage>
    </root>
    <root>
      <mymessage><b>M3</b></mymessage>
    </root>
    --> As you can see, just the last message M3 is send 3 times!
    What can I do?
    Regards Mario

    If I take the payload from SXMB_MONI an try to test, I get an syntax error when I copy&paste the data into the message mapping.
    This is very strange, because
    a) the message mapping is done on basis of imported IDOCs!
    b) the BPM works without throwing a mapping error
    So what should I do?

  • BPM - Par for each

    I am having some issues with my Par for Each block in my BPM.
    My scenario is File(CSV format) --> BPM --> IDOC.
    The BPM will receive the file and it will convert the incoming message into IDOC and in the Parforeach Block I am sending the IDOC to R/3.
    Currently in my file I am having around 1300 Records.
    I am seeing the following error message in the Message Monitoring
    Work Item  000000015782 :Object Flowitem method cannot be executed
    Error When Processing Node 00000000023 (Parforeach index 00000000)
    Parforeach  table element contains  1268 entries
    Error when creating  a component  of type "dynamischer paraller  abschint"
    Error When Processing Node 00000000023 (Parforeach index 00000000)
    Error during result  processing of work  item  00000015784
    Question
    Whats the problem ? Previously when I ran for few records it ran fine? so the Parforeach is unable to handle the load? Where to increase the limit.
    thanks for your help.

    Hi Jenni,
    Check this...
    A ParForEach is recommended if:
    ·        The number of parallel processing branches is less than 999 (the multiline table element that is processed in the ParForEach contains less than 999 lines).
    http://help.sap.com/saphelp_nw04/helpdata/en/ce/bb2c421f3fda2ce10000000a1550b0/content.htm
    Regards
    Anand

  • I'm mixing tracks together and can't work out where the volume and BPM control for each Track is located

    Which Table would be the best for mixing tracks together? I've been off the game for a bit and have forgotten, but last time i made a good mix tape from the New project table....
    Where do i go to match up the BPM for each track i lay to match up?
    How do i get the Volume line to pop up on each track so i can fade accordingly?
    Thank you to those who can help out

    The correct way to target instances m1 thru m10 using bracket notation would be... 
    this["m"+i]
    or even more correctly...
    this["m"+String(i)]

  • Header for alv block list

    Hi experts,
    im trying to build an alv report with block, and after some hours i finally get how it works but the report has 5 blocks .. and 1 header for all the report...and 1 title for each block
    the thing is that for each block theres are their events.. so if i use the TOP OF PAGE that good for each block title, but how can i put a general HEADER for all the report
    its something like this
    Report 0001              DATE
    title 1(top of page)
    alv_list1
    title 2(top of page)
    alv_list2
    title 3(top of page)
    alv_list3
    so... guys im kinda a noobie in alvs so i apreciated any ideas...
    thans in advance

    thx darek,
    but im working with alv LIST blocks .. and each block has top of page and top of list...
    im looking  for a top of list , for say, of all the report, of all the blocks...
    anyone?
    thanks in advance

  • ** Is it possible to create new BPM instance for each record (Multiline)

    Hi friends,
    In my scenario, JDBC adapter (sender) polls the open purchase order items from the table at the specified interval and send to BPM. In BPM, we used transformation step to split the messages to process each PO . The scenario is working fine. The problem is assume that if we process 10 PO, the error is in  4th PO while process, the BPM will be stopped in 4th PO. Once we correct the error, we are able to restart.
    In this case, we are not able to skip the 4th PO and process from 5th PO onwards. ie. the processing is sequential. Instead, we want to start new BPM instance for every PO. Advantage is that if 4th PO is error, only that BPM instance (work item) will be stopped. Remaining 9 POs will be completed.
    So, how do we start new BPM instance for every PO ?
    Kindly tell me, friends.
    Thank you.
    Kind Regards,
    Jeg P.

    Hi,
    There are two ways to achieve this.  In BPM and before BPM.
    Before BPM:
    Use 1 to unbounded mapping and 1 to unbounded interface mapping.
    In your mapping, make sure you create a seperate message for each PO.
    In BPM:
    Create a multiline container with you POs using a 1 to n mapping.
    Now add a ForEach block to loop through the multiline container and send each PO.
    Important:  Add an exception branch to catch any exception for each send so that the exception does not make the BPM fail.
    Regards,
    Yaghya

  • How to process a block for each row in an internal table....

    Hi experts....
    In po approval workflow the scenario is like this.... for each po there may be more than one approver. approvers list i am maintaining in the ztable. list of approvers(no of approvers) is decided by the po value. I have collected these approvers into internal table. now i have to process a block ( approving or rejecting the po... )in the workflow for each row in the internal table.
    how can i do this. based on the decision of the 1st approver  approves the po then it should go to next approver in the internal table...otherwise end the workflow.....
    Please help me......

    i have created an internal table in the workflow container in which i am getting the list of approvers....
    how can i loop the internal table in the workflow...?
    how can i know the index of the loop in the workflow.....(will sy-index work here....? so that i can use loop until step in the main workflow to call the subworkflow..so that if sy-index is greater than no of entires in the itab then i can come out of the loop)

  • Assign payment block Reasen for each Tolerance key

    Dears experts ,
    hi , could you help me to check is it available to assign payment block Reason for each Tolerance key

    Hi,
    Please provide Details of your exactly requirement --
    as per my observation - above mentioned Tolerance key in QM Quality Management -- Payment block we can't assigned
    Thanking you
    Mahesh

  • Conditionally display an icon for each record in a multi record block

    Hi,
    I am using Forms 6i. Is there any way to conditionally display an icon for each record in a multi record block. The SET_ITEM_INSTANCE_PROPERTY builtin does not have many choices. Thanks for your help.

    Henry,
    I doubt that. You would have to replace the text item with an image item. This however can't be done for individual cells in a table but only for the whole column.
    On the web chances are that these could be handled with a custom PJC, but this solution doesn't work in client/server
    Frank

  • How to dump block and identify the bytes stored for each column

    SQL> select header_file, header_block
    2 from dba_segments
    3 where segment_name = 'APARTMENTS';
    HEADER_FIL HEADER_BLO
    4 1692
    1 row selected.
    SQL> alter system dump datafile 4 block 1693;
    Statement processed.
    How can I see the dump block and identify the bytes stored for each column?
    tab 0, row 0, @0x73b
    tl: 125 fb: H-FL lb: 0x1 cc: 4
    col 0: [25]
    52 65 64 77 6f 6f 64 20 53 68 6f 72 65 73 20 41 70 61 72 74 6d 65 6e 74 73
    col 1: [20] 00 54 00 01 02 08 00 00 00 01 00 00 00 01 00 00 00 00 1b 8d
    col 2: [53]
    00 54 00 01 02 0c 00 00 00 01 00 00 00 01 00 00 00 00 1b 8e 00 21 09 00 00
    00 00 00 00 11 00 00 00 00 00 01 45 6d 65 72 67 65 6e 63 79 20 44 65 74 61
    69 6c 73
    col 3: [20] 00 54 00 01 01 08 00 00 00 01 00 00 00 01 00 00 00 00 1b 8f

    SQL> select header_file, header_block
    2 from dba_segments
    3 where segment_name = 'APARTMENTS';
    HEADER_FIL HEADER_BLO
    4 1692
    1 row selected.
    SQL> alter system dump datafile 4 block 1693;
    Statement processed.
    How can I see the dump block and identify the bytes stored for each column?
    tab 0, row 0, @0x73b
    tl: 125 fb: H-FL lb: 0x1 cc: 4
    col 0: [25]
    52 65 64 77 6f 6f 64 20 53 68 6f 72 65 73 20 41 70 61 72 74 6d 65 6e 74 73
    col 1: [20] 00 54 00 01 02 08 00 00 00 01 00 00 00 01 00 00 00 00 1b 8d
    col 2: [53]
    00 54 00 01 02 0c 00 00 00 01 00 00 00 01 00 00 00 00 1b 8e 00 21 09 00 00
    00 00 00 00 11 00 00 00 00 00 01 45 6d 65 72 67 65 6e 63 79 20 44 65 74 61
    69 6c 73
    col 3: [20] 00 54 00 01 01 08 00 00 00 01 00 00 00 01 00 00 00 00 1b 8f

  • IPhone Ad Hoc - One build for block of UDIDs or one build for each UDID?

    Hello.
    For ad hoc distribution, do I need to create a new unique build for each of the UDIDs from my potential testers? Or just one time for the entire set of UDIDs?
    Please set me straight, I've been searching for this answer, but could not find anything.
    Thank you so much.

    You must add each UDID to your distribution provisioning profile in iTunes Connect. Once you have done that, you can use a single .mobileprovision file and a single binary for all provisioned users. You do not need to build a version for each user.

  • Par For each/ForEach

    All,
    Here s my situation:
    I have performed a transformation step 1:N: where i split my messages N times.
    After which i am sending my N messages one by one to the receiver.
    Now should i use a Parfor each or a ForEach for this scenario???
    In either way how should i define my parameters.My source is OrderRequest and my target is OrderResponse(N)
    in my container step i defined these msg types
    SingleOrderResponse TYPE: OrderResponse_ABS and MultiOrderResponse TYPE: OrderResponse_ABS and  now i tried Parforeach in the trasformation step of my BPM:i specified my interface mapping gave source msg as OrderRequest
    and target msg as MultiOrderResponse checked the multiline container element,and next is my send step which i included in ParForEachBlock, where i specified my multiline element as MultiOrderResponse and in the currentline i specified singleOrderResponse and in the stpe step i used the singleOrderResponse Msg type.
    But in my tranformation step, i have this error msg saying cannot define multiline element....
    Can anyone suggest me on what i should do?
    Thanks in advance

    Hi Aarthi,
    Let me first make sure that I have your requirements right.
    What you want to do is perfrom a 1:N transformation and then send each of your response to the receiver.
    For this , in your BPM,
    1. the first step will be receive step where you receive your request message.
    2. the next step will be your Transformation step, where you perfrom 1:N mapping.
    3. Finally, you will have to define a block with a send step. the bloack can be par for each or for each.
    From what I understood of your definition of the problem, i think you have put your transformation step within the block and that should not be done.
    Also, with the transformation step, the containder element for the reponse should be a MULTILINE element as the mapping will produces N messages.
    DO let me know if i have understood your requirements well and if this solution does help you.
    Regards,
    Bhavesh

Maybe you are looking for

  • How to make a Transparence Background GIF Animated??

    Hi, How to make a Transparence Background GIF Animated?? Any Special Pro software do i need like Photoshop ? Posible to use Keynote or something like that? Thanks

  • Flash Player 10.1 Won't register

    I went to log on to www.Hulu.com and the site that I needed to download the latest verson of Flash Player. I clicked the download and install and got an error message: Could not register Active X controls. I am logged on to the computer as the admins

  • Configuration to send the smartform through fax

    Hi, I have used CONVERT_OTF_AND_FAX and SO_OBJECT_SEND FM's to send the smartform through fax.After executing SO_OBJECT_SEND function module,I am getting sy-subrc alue as 9(OBJECT_NOT_SEND).I am able to send the document through fax.But when I click

  • Menu deformation perspective photoshop cc 14.2 greyed

    why is menu deformation perspective photoshop cc 14.2 greyed ? I use last update of photoshop cc on mac os 10.9, the image is RVB 16 bits

  • Itunes mac automatically opens, due to bluetooth?

    i've read how itunes can automatically opens when iphone/ipods are connected to a Mac, but itunes on my rMBP is opening periodically for some other reason. i suspect it may have something to due with bluetooth connecting to an external stereo? even t